:10000000C8080020C5000000C1000000C1000000B9
:1000100000000000000000000000000000000000E0
:10002000000000000000000000000000C10000000F
:100030000000000000000000C1000000C10000003E
:10004000C1000000C1000000290F0000350F0000B2
:10005000C1000000C1000000C1000000C10000009C
:10006000C100000001100000C1000000C10000003C
:10007000C1000000C1110000C1000000C10000006B
:10008000C1000000C1000000C1000000C10000006C
:10009000C1000000C1000000C1000000C10000005C
:1000A000C1000000C1000000C1000000C10000004C
:1000B000C1000000C1000000C1000000C10000003C
:1000C000FEE70000002370B50A480B490B4C1A18D4
:1000D0008A4203D2E55804331560F8E70021084B43
:1000E000084A934201D202C3FBE701F055FB00F03E
:1000F000FBF870BD000000200C0000201C2F000049
:100100000C000020C404002010B5162059248821BA
:10011000034B5C60586059605A68002AF9D010BDE2
:10012000FC0000502122064BDA60203A58609960AA
:100130001A61BFF36F8F1A69002AFCD17047C0465D
:1001400000C000500022074BDA6058609A6001320C
:100150001A61BFF36F8F1A69002AFCD1014B9868AE
:100160007047C04600C000502222054BDA60213A99
:1001700058601A61BFF36F8F1A69002AFCD170476B
:1001800000C00050FA22534B520030B51A600328C9
:1001900000D99EE0504D514C514A524B02F0D8FDCF
:1001A00002254C71642000290DD029784843A060B5
:1001B0000F2091688143916091680B3801439160F1
:1001C0001A78012121E029784843E06007209168EE
:1001D00081439160916801300143916002211A7856
:1001E0000A431A701A78013971E06420002911D08D
:1001F0006978484320600320916881439160916849
:1002000002380143916004211A780A431A701A785F
:1002100049185CE069784843606001209168814337
:100220009160916800180143916008211A780A438F
:100230001A701A7804394AE06420002910D0A9788D
:10024000484320613F2091688143916091682F3835
:10025000014391601A78202102431A701A7836E01F
:10026000A978484360611F2091688143916091683B
:100270000130014391601A78102102431A701A78F4
:1002800025E06420002911D0E9784843A061FF20CF
:100290009168814391609168BF38014391601A78F9
:1002A00002431A707F2219780A4011E0E978484326
:1002B000E0617F2091688143916091680130014342
:1002C0009160020019780A4340211A701A788A4313
:1002D0001A7030BD8001002077000020240000202B
:1002E000804000507600002055233749F0B5374C48
:1002F0000B60153B23603648364B374E0360374B57
:10030000374A3360374B85B01360002383608B60BE
:100310000821A360B1609360FFF7F6FE0123324D20
:100320002A681A432A60314A0294E968194202D1C4
:10033000013A002AF9D1002380222B612B6A520254
:10034000134304222B622A4B2B62284BE96811428B
:1003500002D1013B002BF9D102232B61254BAB606D
:1003600080239B026B6101F0CBF9234B1A68234B6E
:100370005A43234B5A6000229A6005321A60802249
:10038000520219681142FCD00122F8201D4C400293
:10039000236813432360FFF7D5FE01941A4F1B4CCB
:1003A0005B3039D11A48FFF7CDFE38601948FFF7A6
:1003B000C9FE030EE370030CDBB2A370030ADBB2C9
:1003C000C0B26370207033E00040005040400050E5
:1003D0008040005055550000C0400050CF5F0000E5
:1003E00000410050F50F00000002005091D00300C2
:1003F000174200001C0002100800002020A1070086
:1004000010E000E000C000508C02002077000020C7
:1004100004F0010008F00100F8204002FFF7A4FEFC
:1004200001235B423B600433E370A370637023706D
:10043000F924F14F64022000FFF784FEEF4B010E18
:10044000E218EF4B04349954020C3A70020A7A70A5
:10045000EC4AB87004379442EDD11A78FF2A03D1E0
:10046000DF3A1A7000225A700124E748FFF76AFE4B
:100470009521019B019A1B680002A3431360E34B83
:10048000000A18601A680906521800211A60E04A2A
:10049000802711700021DF4ABF0111701B68DE4AFE
:1004A000DBB21370DD4A13701F2311780B401370F9
:1004B000DB4A13683B431360FFF726FEA021C023ED
:1004C000C9051B014B63C0239B000B63D54AD64B68
:1004D000F0205A620B22DA60083A1A63852212026F
:1004E000DA629A6882439A6000221A615A6822434B
:1004F0005A60C322920094466046CC4B1F609F58BE
:10050000CB4A17401F500820B769B761F769074306
:10051000F7611860C020C02780001E583F063602D1
:10052000360A3E431E5080260138FF381860C14805
:10053000F6040660C04E0660C04E4660C2208000D1
:100540001E5832408026F60132431A50AA69BC4B2D
:10055000FF201340C022D2021343AB61C023029A92
:100560009B0253604B6BB74A23434B6309231362CF
:10057000516A536A814323430B435362146300223D
:10058000B14B5A600393A64D2B685B072ED5FFF73E
:10059000BBFDF920F926019B019A1B684002234309
:1005A0001360FFF7E1FD944F7602944B944AF318E1
:1005B000D15C3B7809061B04C9187B7830001B020C
:1005C000C918BB780436C918FFF7ACFD8D4B04374A
:1005D0009E42EAD1019B019A1B68A343136000234A
:1005E000039A536004222B6893432B6008262B68E0
:1005F00033422ED0FFF788FDF820019B019A1B683B
:10060000400223431360FFF7AFFD5B21F82049420E
:100610004002FFF787FD8D4B8D481968FFF782FD7B
:100620008C48C178827843780906B3401204007878
:100630008A18D11809188848FFF774FD019B019AA0
:100640001B68A34313600023039A53602B68B343D2
:100650002B606F4B1B78032B00D029E2704A136884
:100660009B0155D413685B0352D5136823424FD0C6
:10067000802315685B041D404AD11368A3431360AF
:10068000764B1B78002B43D0802106261368C904C3
:100690000B431360724B1878C0B2411CC9B2197079
:1006A00070490E541878C0B2461CF6B21E7005266A
:1006B0000E541878C0B2461CF6B21E700D5418784D
:1006C000C0B2451CEDB21D70674DAC4667462D7833
:1006D000EDB26E1CF6B23E700D541878C0B2451CD7
:1006E000EDB21D7086250D541878C0B2451CEDB2D0
:1006F0001D7004250D541878C0B2451CEDB21D7054
:10070000564B1B78DBB20B541168584B0B401360EF
:1007100001F0EAF8FF2256490B68134200D1ADE020
:100720003F4803685B0300D4A8E0802306685B04AD
:100730001E4000D0A2E0802209270B68D204013BB2
:100740000B60036813430360454B1D78EDB26A1CD0
:10075000D2B21A70434A57551D78EDB26F1CFFB2E2
:100760001F70082757551D78EDB26F1CFFB21F7020
:1007700056551D78EDB26E1CF6B21E703A4E0295BB
:10078000B44665463678F6B2771CFFB22F70029DEC
:1007900056551D78EDB26E1CF6B21E70B826565531
:1007A0001D78EDB26E1CF6B21E7003260F683E4037
:1007B0007F2756551E78F6B2751CEDB21D700D6878
:1007C000BD43EDB295551D78EDB26E1CF6B21E70AC
:1007D000022656551D78EDB26F1CFFB21F708027A0
:1007E00057551D78EDB26F1CFFB21F705655026849
:1007F0001E4B1340FF223DE092020020000EFEFF40
:100800009102002018F20100FC0F100018000020D7
:10081000C104002014000020850200207D0100207A
:10082000AC0200201600003F0000154000E100E08F
:10083000FF00FFFF2000014000000168442F00007E
:10084000FFFF00FF00000E40FC0000508C02002063
:1008500004F001007700002008F00100B904002036
:100860006C0000208401002084020020FFFFFFFBB9
:10087000B404002003600B6893430B60FF23DE4940
:100880001B020A681A4200D112E1DC4B1A685203BB
:1008900000D40DE1802218685204104000D007E116
:1008A000802509261A68ED042A431A60D44B1D7866
:1008B000EDB26A1CD2B21A70D24A56551D78EDB20A
:1008C0006E1CF6B21E70082656551D78EDB26E1CD1
:1008D000F6B21E7050551D78EDB26E1CF6B21E7049
:1008E000C94E0295B44665463678F6B2771CFFB21B
:1008F0002F70029D56551D78EDB26E1CF6B21E701B
:10090000B8265655C0260D68B600354224D01D784D
:10091000EDB26F1CFFB21F70505508683040B042F6
:100920000CD119780325C9B2481CC0B21870FF2039
:100930005054B6480178A943017009E01878C0B254
:10094000451CEDB21D700968090A0139C9B211547C
:10095000A948AF49056828E0C02508682D0128424C
:1009600026D01878C0B2461CF6B21E70145408681F
:100970002840A8420CD119780C25C9B2481CC0B235
:100980001870FF205054A1480178A943017009E074
:100990001878C0B2451CEDB21D700968890A01398A
:1009A000C9B2115494489B4905682940016065E02B
:1009B000C0250868AD01284225D01878C0B2461C71
:1009C000F6B21E700226165408682840A8420CD1C0
:1009D00019783025C9B2481CC0B21870FF20505495
:1009E0008A480178A943017009E01878C0B2451C13
:1009F000EDB21D700968090B0139C9B211547E4866
:100A000085490568D1E7C0270E681D783F023E4042
:100A10008248EDB2002E21D06E1CF6B21E70032665
:100A200056550D683D40BD420CD11978C9B24D1CD8
:100A3000EDB21D70FF2555543F21744D2E78314085
:100A4000297009E01D78EDB26E1CF6B21E700968BF
:100A5000890B0139C9B2515567490CE06F1CFFB2CF
:100A60001F7056551D78EDB26E1CF6B21E70674EA3
:100A70003678264056550D68284008601978C9B266
:100A8000481CC0B21870022050541978C9B2481CD2
:100A9000C0B21870802050541978C9B2481CC0B236
:100AA000187006235354554A5D4B11680B40136070
:100AB0005C4B52491B680A68234200D115E25A4830
:100AC000524B5A4E5A4D844692043BD537682A6899
:100AD00008680292020057481040029A08605200CB
:100AE0000021D71903225448574001604248534A15
:100AF000FFB201601F701168514A126818785200E5
:100B000052180C2192004A400243D2B21A704D4A48
:100B100011684D4A1268187852005218302112019B
:100B20004A400243D2B21A70484A116862461268BB
:100B30001878520052184021920149424A4002431B
:100B4000D2B21A7031682A6852005218D2B2002A02
:100B500001D0032A14D103221978114210D03C4A43
:100B60001168002903D1F531FF3111607CE0126872
:100B7000042A79D8C020204980000A68024372E024
:100B8000197821421ED0022A12D0314A1268002A56
:100B90006AD18020184940000A6802430A60022195
:100BA000254A14601A78A2431A701A780A4320E082
:100BB000114A17491068014011601168FF221202A2
:100BC0000A404DE00221187808424DD0012A41D058
:100BD0001F4A1268002A47D180250748AD000268E5
:100BE0002A430260144A14601A788A431A701A78E9
:100BF00022431A7038E0C046B4040020AC02002042
:100C00006C00002084010020840200207600002077
:100C1000FFFCFFFFFFF3FFFFFFCFFFFFFF3FFFFFE3
:100C2000FFFFFFFB8C0200201042005030420050BA
:100C300034420050FFDFFFFF804200503842005036
:100C40003C4200501C4200501842005014420050D8
:100C500080010020A74AA84910680140116012686D
:100C6000002A01D1A5490A60A54AA6491268096867
:100C700049008918C9B2002901D0032915D10C22D5
:100C80001978114210D0A04A1168002903D1F5311A
:100C9000FF3111604EE01268042A4BD8C0209549FC
:100CA00000010A68024344E003210422187810423C
:100CB0001DD0022911D09449096800293AD1802514
:100CC0008C48ED000168294301608C490C6019785B
:100CD000914319701A7808211FE0864A8B491068E1
:100CE000014011601168FF2212020A401EE0082034
:100CF0001D7805421ED0012912D0834909680029B8
:100D000018D180267B4D36012968314329607B4903
:100D10000C6019788143197019780A431A7009E038
:100D2000744A7A491068014011601268002A01D1A2
:100D300072490A60764A7749126809684900891839
:100D4000C9B2002901D0032915D1302219781142E6
:100D500010D06D4A1168002903D1F531FF311160BF
:100D60004EE01268042A4BD8C020624980010A680C
:100D7000024344E003211022187810421DD00229BA
:100D800011D06149096800293AD1802559486D017F
:100D900001682943016059490C6019789143197021
:100DA0001A7820211FE0534A5B4910680140116006
:100DB0001168FF2212020A401EE020201D78054221
:100DC0001ED0012912D050490968002918D1802667
:100DD000484DB60129683143296048490C601978AB
:100DE0008143197019780A431A7009E0414A4A4947
:100DF0001068014011601268002A01D13F490A6061
:100E0000464A11686246126852005218D2B2002A4D
:100E100001D0032A18D13F211A788A4313D03A4BC4
:100E20001A68002A04D1F532FF321A60FFF7ABFBD3
:100E30001B68042B01D9FFF7A6FBC0212D4A09022C
:100E400013680B434EE003224021187808421FD05C
:100E5000022A13D02C4A1268002A01D0FFF793FB14
:100E600080252448ED0102682A430260234A146069
:100E70001A788A431A701978802224E01D4B284A78
:100E800019680A401A601A68FF231B02134024E005
:100E9000187840B2002801DBFFF775FB012A16D055
:100EA000194A1268002A01D0FFF76DFB802511480E
:100EB0002D0202682A430260104A14607F221878CB
:100EC00002401A701A780A431A70FFF75CFB094B4C
:100ED000134A19680A401A601B68002B01D0FFF7FB
:100EE00052FB064A1360FFF74EFB0E4B13400B609C
:100EF000FFF749FBB4040020FFFCFFFF80420050D5
:100F0000384200503C42005080010020FFF3FFFFB8
:100F10001C42005018420050FFCFFFFF1442005007
:100F2000FF3FFFFFFFDFFFFF0422014B1A62704704
:100F3000C040005008222A4B70B51A62294B1A682B
:100F400052034BD580201A6880020240264903D103
:100F50000A601A68024304E000220A601968234A02
:100F60000A40802105241A601A68C9040A431A60DD
:100F70001F4A204E1078C0B2411CC9B211701E49E0
:100F80000C541078C0B2441CE4B2147004240C5405
:100F90001078C0B2441CE4B2147000240C541078D1
:100FA000C0B2441CE4B214703478E4B2651CEDB2F3
:100FB00035700C541078C0B2441CE4B2147087240D
:100FC0000C541078C0B2441CE4B214701A68920336
:100FD000D20F0A541968094A0A401A6070BDC04607
:100FE000C0400050AC0200207C420050FFFFFDFFDB
:100FF0006C0000208402002084010020FFFFFFFB22
:10100000F7B50122584B59499A600B680091002BA3
:1010100002D00B68013B0B60002001250200544CFC
:1010200023680194534E9700BF59002F57D0802159
:10103000514F09013C6A0C433C62396B2942FCD098
:101040004D4F4E493F68BFB20F600F68FA2F04D969
:101050005F1C0120322B03D904E0002B2DD11F008F
:101060003B002CE00020464B9860464B072A1FD8D7
:10107000100001F06DFE08041D0B120E19158021E1
:101080001868084318601868284310E01868802121
:101090000CE080211868084318601868022105E0F8
:1010A00080211868084318600321186808431860F5
:1010B0001868013018603B0000E0013B01209100FE
:1010C0007758013F7750002F09D12C009440FA2126
:1010D0002B4F4900BE68A643009CBE6021600132D0
:1010E000082A9FD1002801D0019A1360264A274878
:1010F000138801339BB213800378002B21D0244B3B
:101100001968013119601968C8239B00994218D9E0
:10111000204B19680F230B401F4940330B700023ED
:101120001E4903701E480B7003701E4803701E4852
:1011300003701E48037006200B701D4988601D490E
:101140000B601D4B1B689B030DD5FF2311881940B5
:10115000802903D10122194B1A6004E01288134040
:1011600001D1164A1360F7BD200001408001002024
:101170000C0000202400002000000E407000002021
:1011800080400050B4040020AA020020C1040020C6
:10119000BC040020180000207D0100206E0000200B
:1011A000B2040020C20400206C000020BB04002018
:1011B0000000154020000020AC0200207C420050BE
:1011C000F0B50825D94B85B01A6802A9D2B207310B
:1011D0000A7098691F00284000D148E19A697F246D
:1011E0002A439A614022087810400A782240002859
:1011F00000D19EE07D2A00D189E07E2A00D089E0DE
:10120000CB4B1A78002A6ED1CA4A1378DBB2002B76
:1012100002D01378013BE9E00B22C74CC74922708A
:10122000013A6270E632A370E3702271EC3A6271A7
:101230003A32A371E2710A680126120E22720A681C
:10124000120CD2B262720A68120AD2B2A2720A6890
:101250000C21D2B2E272BA4A1170BA4A1370BA4A79
:1012600013711022FB681343FB60FB689218134351
:10127000FB60FB681D43FD602578EDB23D602800F2
:1012800000F00EFB80221204AE4217D88022BB6908
:1012900012041342FAD1AB4AA44913780136013340
:1012A000DBB21370E35CF6B2DBB20B601378DBB237
:1012B000E35C5840C0B200F0F3FAE3E7BB691340C7
:1012C000FCD19A4A9F4910600A780132D2B20A7062
:1012D0009E4A974913709E4A136002220A709D4AE3
:1012E00013609D4A42E01B78022B00D0F1E100F030
:1012F000C9FA904B18701A78002A00D0E9E18F4A99
:101300001268D2B21A700F2219780A400CE100223A
:101310008F4B9DE0914A1368002B00DBBAE1136804
:101320005B005B081360894A1378013BDBB21370E2
:10133000B0E1002A1CD18024844964000B78DBB220
:10134000581CC0B2087086485B001C520B785B00CA
:101350001A520B787C4ADBB213710B788021814AD8
:10136000DBB213707D4A090613680B431360B0E1CA
:101370006F4A1278D2B2022A6CD0032A00D089E1D7
:10138000794A0C7811781F2222408A4200D0A0E1CD
:101390006F4C724A206011680194490100D598E1B0
:1013A00010687249014011601021DA680A43DA605E
:1013B000DA6849180A43DA60DA6861491543614A14
:1013C000DD60147808781500844206D1802299697E
:1013D00012040A4000D07CE13AE013785648DBB2B0
:1013E000C45CE4B2231F3B2B03D90B78DBB2137030
:1013F0006FE13C60200000F053FA01268022BB69B7
:1014000012041342FAD12B784B4A0133DBB22B7012
:10141000D35C4649DBB20B602B780136DBB2D35C80
:10142000F6B25840C0B200F03BFAB442E6D2802295
:1014300012048023B9691B041142FAD13B4A10609F
:10144000BA691A40FCD12B780133DBB22B70019BB7
:101450001A603EE101223C4B1A713F4A1368591C45
:101460001160632B00D915E1394B186012E13B4A3A
:10147000364C13683A4D002B00DBF6E02378DBB2E4
:101480005A1CD2B222700A785B00EA522E4A1379B3
:1014900001925B00EB5A002B00D1FBE013795B005B
:1014A000EA5A019B1B79217802339B18DBB28B42ED
:1014B00000D0EFE023780600DBB25A1CD2B22270D3
:1014C00080225B009200EA52244B244A1B685B0096
:1014D0005B0813601C4A137994465B00EB5A013396
:1014E000B3420FDB1379224AF318DBB25B00EB5AED
:1014F000DBB29355935D01365840C0B200F0D0F98D
:10150000F6B2E7E70A4A1378DBB2022B06D0032BC8
:1015100000D0BFE000220E4B1A60BBE0002829D0AB
:1015200000231370FF22034B1A70D2E00000154015
:10153000C10400207D01002084010020180000204B
:101540006C000020C00400200C000020BB04002020
:10155000BC040020B404002020000020AC020020C5
:10156000B2020020C20400207C010020FFFFFFFE29
:101570007C000020584B19001A79702A35D10022BE
:10158000564D57482A609446597A0268120E914285
:1015900000D07FE0FF219E7A0268120C0A4096423A
:1015A00078D1DE7A0268120A0A40964272D11A7B1A
:1015B0000068084082426DD103224A4802705B797C
:1015C000494ADBB213701378DBB2634501D1037073
:1015D0002BE063462B602378444ADBB21370444B04
:1015E0001A68444B1340424A53E01A79722A1FD1B9
:1015F00000243A4A3A481460597A0268120E91421D
:1016000048D1FF219D7A0268120C0A40954241D1CF
:10161000DD7A0268120A0A4095423BD11A7B0368C0
:101620000B409A4236D12F4B1C70334B197050E04F
:101630001D7818785A78EDB2013290422ADD5A7836
:1016400001980132D2B2027100791A78121AD2B21C
:101650001A7000220132D0B285428DD960460079DD
:101660008018085CC0B28854F4E72378013B5B0023
:10167000E85A80235B0098420CD12378DBB2581CD7
:10168000C0B2207009785B00E95280211368090616
:101690000B431360BB69194A1B0403D502239168ED
:1016A0000B4093600122B969144B114206D099692D
:1016B0000A409A61022299680A409A60BB699B06B7
:1016C00003D40E4B9B69DB0603D50223BA68134093
:1016D000BB6005B0F0BDC0467C000020BC0400200B
:1016E00018000020C10400207C010020C20400205A
:1016F000AC020020FFFFFBFF7D0100200000154031
:1017000073B51E4D01AE04222900300001F0B6FB76
:10171000A0221B4CD202236A0020134215D11A03C7
:1017200001D4184800E018489A030ED4DA05D20D07
:101730000232800850431A04920F9B04B15CDB0E06
:101740000233594301F00EFB800007230F4E306037
:1017500022691340022B02D09B00ED1868680F230A
:10176000A1691940013101F0FDFA094B7060094986
:10177000C01801F0F7FAB06073BDC046F82E000043
:1017800000020050001BB700008051010000002043
:1017900020A1070040420F000022174B30B51A600D
:1017A000164B073219690A400AD10421144A1A62F9
:1017B000144AD86808420FD1013A002AF9D10BE047
:1017C000072A18D10421104A1A62104AD868084220
:1017D00002D1013A002AF9D15924162088210C4A55
:1017E0005460506051605568002DF9D002221A6192
:1017F0000022074B5A6030BD00000020000200505C
:1018000017420000E12E000039560800675600001C
:10181000FC00005010B5162059248821034B5C6051
:10182000586059605A68002AF9D010BDFC00005079
:101830002122064BDA60203A586099601A61BFF3A2
:101840006F8F1A69002AFCD17047C04600C0005053
:101850000B4B1A7819785200D2B24A4052001978CC
:10186000D2B24A4012011978D2B24A401978D2094C
:1018700049005218D2B21A701878C0B27047C046E8
:101880008502002010B5FFF7E3FF0F23034A18403D
:101890001378C0181F231840107010BD14000020CA
:1018A0000023C20700D55E33820701D5BC22534016
:1018B000420701D561225340020701D5C22253409D
:1018C000C20601D59D225340820601D523225340F2
:1018D000420601D54622534040B2002801DA8C224C
:1018E0005340180070470000F0B5D04BD04C1A7828
:1018F000237893B09A4201D101F009FA802322782B
:10190000CC4D5B00002A12D1FF32FF32AA5A1900D7
:101910009A4202D18022520015E02378DBB25A1C91
:10192000D2B222705B00EB5A8B42F6D1F2E72278FA
:10193000013A5200AA5A9A42ECD02278D2B2511CF3
:10194000C9B22170F5E723785B00EB5A934204D1CA
:1019500023780133DBB22370F5E723785B00EB5A81
:10196000002B01D101F0D3F923785B00EB5A02334D
:10197000DBB20193019A2378D318DBB25B00EA5AF9
:1019800080239B009A4201D001F0C1F9002630006B
:101990002378019AD318DBB25B00EE52019AF3B2BE
:1019A0009A420FD92278D2B2531CDBB22370520074
:1019B000AA5AD3B202AA93554340D8B2FFF770FF98
:1019C0000136EBE723780133DBB22370002848D0DF
:1019D000994B02AA1B7892789A4242D100200624A1
:1019E000964B974E18701978C9B24A1CD2B21A7029
:1019F000944A54541978C9B24C1CE4B21C700524A2
:101A000054541978C9B24C1CE4B21C705054197863
:101A1000C9B24C1CE4B21C703478E4B2651CEDB25F
:101A2000357054541978C9B24C1CE4B21C70862429
:101A300054541978C9B24C1CE4B21C70022454549A
:101A40001978C9B24C1CE4B21C7002AB1B79535418
:101A50007D4B7E4A186011687D4B0B40136001F08E
:101A600056F90125744A02AB9E78137814009E4201
:101A700016D1784B1978FF2901D1002119701878F7
:101A800002A909790130884209D01878724FC0B292
:101A90003870002903D06D4F3868284338601970BA
:101AA00013789E4201D001F0E3F88021674AC9040F
:101AB00013680B43136002AB5B790F2B01D101F06C
:101AC0007DF800D99FE0072B00D1FEE144D8032B1D
:101AD00000D190E137D8012B00D14DE1022B01D08C
:101AE00001F0C6F80620554B554F1978C9B24A1C6B
:101AF000D2B21A70534A50541978C9B2481CC0B2B5
:101B00001870052050541978C9B2481CC0B218701A
:101B1000002050541978C9B24C1CE4B21C703C78B7
:101B2000E4B2661CF6B23E7054541978C9B24C1C2B
:101B3000E4B21C70832454541978C9B24C1CE4B22A
:101B40001C700724F9E2052B00D15EE100D9FDE20B
:101B50001168424B0B4055E10A2B00D1CEE318D857
:101B6000082B00D129E3092B01D001F081F80023D3
:101B700080213B4A890113603A4AD1673A4AFF21E2
:101B80001370FA22394BD2001A60394A117001F0F1
:101B90005BF80C2B00D180E300D253E30E2B01D075
:101BA00001F066F80620254B254F1978C9B24A1C6A
:101BB000D2B21A70234A50541978C9B2481CC0B224
:101BC0001870052050541978C9B2481CC0B218705A
:101BD000002050541978C9B24C1CE4B21C703C78F7
:101BE000E4B2661CF6B23E7054541978C9B24C1C6B
:101BF000E4B21C70862454541978C9B24C1CE4B267
:101C00001C7050549AE2182B01D100F061FF6AD881
:101C1000122B00D1DFE32DD8102B00D19FE3112B25
:101C200001D100F0FFFB01F023F8C046BB04002007
:101C3000C2040020B20200207C0100206C000020C1
:101C40008402002084010020BC040020AC0200209B
:101C5000FFFFFFFBA9020020B9040020FFFFFBFFEC
:101C60007C42005004E100E0C1040020800100201B
:101C70007D010020142B01D100F038FF01D200F0CB
:101C800083FC152B01D000F0F3FF05201168E14B18
:101C9000E14F0B401360E14B1978C9B24A1CD2B234
:101CA0001A70DF4A50541978C9B2481CC0B2187073
:101CB000042050541978C9B2481CC0B218700020D2
:101CC00050541978C9B24C1CE4B21C703C78E4B290
:101CD000661CF6B23E7054541978C9B24C1CE4B27A
:101CE0001C70942429E2392B01D100F087FD09D81A
:101CF0001A2B3CD000D22DE1382B01D100F0C5FCCD
:101D000000F0B6FF3B2B01D100F04BFE01D200F0FA
:101D1000FCFD712B01D000F0ABFF0420BF4BBE4E89
:101D20001978C9B24A1CD2B21A70BD4A50541978F7
:101D3000C9B2481CC0B21870032050541978C9B2F7
:101D4000481CC0B21870002050541978C9B2481C01
:101D5000C0B218703078C0B2441CE4B23470505431
:101D60001978C9B2481CC0B21870F123DEE002AB8A
:101D7000197AAC480023DCE004200626AA49C8678B
:101D8000A6490C78E4B2601CC0B20870A44806559D
:101D90000C78E4B2661CF6B20E70052606550E7875
:101DA000F6B2741CE4B20C70002484550E78F6B2BE
:101DB000771CFFB20F7084550E78F6B2771CFFB215
:101DC0000F70812787550E78F6B2771CFFB20F701F
:101DD000FE2787550E78F6B2771CFFB20F70AF2141
:101DE00081558D490B7091490C7091490C701168A7
:101DF00099430B0006E004218E4B19608021136883
:101E0000C9020B43136000F033FF0B20834B824F5A
:101E10001978C9B24A1CD2B21A70814A5054197842
:101E2000C9B2481CC0B218700A2050541978C9B2FF
:101E3000481CC0B21870002050541978C9B24C1C0C
:101E4000E4B21C703C78E4B2661CF6B23E705454A6
:101E50001978C9B24C1CE4B21C708424545419780B
:101E6000C9B24C1CE4B21C7055541978C9B24C1C50
:101E7000E4B21C7050541978C9B2481CC0B2187032
:101E80003E2050541978C9B2481CC0B218706A4834
:101E90000468240E54541C78E4B2611CC9B2197051
:101EA0000168090CC9B211551C78E4B2611CC9B2B1
:101EB00019700168090AC9B211551978C9B24C1CC8
:101EC000E4B21C70036800F0CCFD0520534B524E69
:101ED0001978C9B24A1CD2B21A70514A50541978B2
:101EE000C9B2481CC0B21870042050541978C9B245
:101EF000481CC0B21870002050541978C9B2481C50
:101F0000C0B218703078C0B2441CE4B2347050547F
:101F10001978C9B2481CC0B2187082205054197880
:101F2000C9B2481CC0B2187002AB9B79535400F080
:101F30009FFEDCB2A14205D902AE9C19647AC4545A
:101F40000133F6E700234354042102ABDD7113682B
:101F50000B43136002ABD87900286FD00023314ABD
:101F6000D15CD8B2002903D00133182BF8D1180066
:101F70002A4BC41D1978E4B2C9B24A1CD2B21A70F5
:101F8000274A54541978C9B24C1CE4B21C70841D01
:101F9000E4B254541C78E4B2611CC9B21970002137
:101FA00011551C78E4B2661CF6B21E701A4EB44687
:101FB00061463678F6B2771CFFB20F7016551C7862
:101FC0000021E4B2661CF6B21E70952616551C78E8
:101FD000144FE4B2661CF6B21E70115500211C7835
:101FE000E4B2661CF6B21E7015551C78E4B2661C8D
:101FF000F6B21E701055CCB2844201D300F038FE08
:102000001C78E4B2661CF6B21E707E5C0131165577
:10201000F1E7C046FFFFFFFD840200206C000020B6
:10202000840100209102002004E100E0B9040020B6
:10203000A902002000E100E0180000201224F24B69
:10204000F24F1978C9B24A1CD2B21A70F04A5454ED
:102050001978C9B24C1CE4B21C701124545419787C
:10206000C9B24C1CE4B21C7050541978C9B24C1C53
:10207000E4B21C703C78E4B2661CF6B23E70545474
:1020800019784426C9B24C1CE4B21C7095245454EF
:102090001978C9B24C1CE4B21C7050541978C9B2FA
:1020A0004C1CE4B21C7050541978C9B2481CC0B220
:1020B00018700B2050541978C9B2481CC0B218705F
:1020C000572050541978C9B2481CC0B218705654E1
:1020D0001978C9B2481CC0B218702D205054197814
:1020E000C9B2481CC0B21870332050541978C9B214
:1020F000481CC0B21870342050541978C9B2481C1A
:10210000C0B218702E2050541978C9B2481CC0B201
:102110001870422050541978C9B24C1CE4B21C709B
:10212000692454541978C9B24F1CFFB21F70565419
:102130001978C9B24E1CF6B21E7054541978C9B23F
:102140004C1CE4B21C70505400F092FD0720AE4BC2
:10215000AE4F1978C9B24A1CD2B21A70AC4A505468
:102160001978C9B2481CC0B21870062050541978AA
:10217000C9B2481CC0B21870002050541978C9B2B6
:102180004C1CE4B21C703C78E4B2661CF6B23E70A3
:1021900054541978C9B24C1CE4B21C7085245454B0
:1021A0001978C9B24C1CE4B21C7055541978C9B2E4
:1021B0004C1CE4B21C7000F0E7FC8021136889021B
:1021C0000B4207D01168934B0B4000211360924BD8
:1021D000196002E013680B43136005248A4B8B4F90
:1021E0001878C0B2411CC9B2197089490C541878CA
:1021F000C0B2441CE4B21C7004240C541878C0B261
:10220000441CE4B21C7000240C541878C0B2441C66
:10221000E4B21C703C78E4B2661CF6B23E700C541A
:102220001878C0B2441CE4B21C7087240C5418788F
:10223000C0B2441CE4B21C7013685B0C2B400B54FE
:1022400000F016FD0520704B704E1978C9B24A1C7B
:10225000D2B21A706E4A50541978C9B2481CC0B232
:102260001870042050541978C9B2481CC0B21870B4
:10227000002050541978C9B2481CC0B21870307888
:10228000C0B2441CE4B2347050541978C9B2481C2E
:10229000C0B21870882000F077FC05205A4B5B4EC6
:1022A0001978C9B24A1CD2B21A70594A50541978D6
:1022B000C9B2481CC0B21870042050541978C9B271
:1022C000481CC0B21870002050541978C9B2481C7C
:1022D000C0B218703078C0B2441CE4B234705054AC
:1022E0001978C9B2481CC0B218708B2050541978A4
:1022F000C9B2481CC0B21870FF2317E60520424B34
:10230000424E1978C9B24A1CD2B21A70404A50548F
:102310001978C9B2481CC0B21870042050541978FA
:10232000C9B2481CC0B21870002050541978C9B204
:10233000481CC0B218703078C0B2441CE4B234708B
:1023400050541978C9B2481CC0B218708A20505431
:102350001978C9B2481CC0B218708023E6E5802104
:102360000527136889050B431360274B1978C9B2F9
:102370004A1CD2B21A70264A57541978C9B2481C5E
:10238000C0B21870042050541978C9B2481CC0B2A9
:102390001870002050541978C9B2481CC0B2187087
:1023A0001A48844666460078C0B2441CE4B23470D1
:1023B00050541978C9B2481CC0B2187092205054B9
:1023C0001978C9B2481CC0B2187057540022134B78
:1023D0001A7000F04DFC02AB9A79104BFC2A0ED01B
:1023E00005D8282A0DD0292A1AD1032219E0FD2A5E
:1023F00003D0FE2A14D1042213E0002211E01D7044
:1024000010E002220DE0C0466C0000208402002093
:1024100084010020FFFFFDFF7C42005012000020DD
:1024200091221A7006200526EC4BED4F1978C9B29F
:102430004A1CD2B21A70EB4A50541978C9B2481CDF
:10244000C0B2187056541978C9B2481CC0B218707E
:10245000002050541978C9B2481CC0B2187038789E
:10246000C0B2441CE4B23C70DF4C505421780429C3
:1024700072D8080000F06CFC03182D425800187840
:10248000C0B2461CF6B21E70902616541878C0B220
:10249000461CF6B21E70FD2616541878C0B2461CB3
:1024A000F6B21E7008236BE01878C0B2461CF6B274
:1024B0001E70902616541878C0B2461CF6B21E70D4
:1024C000FC2616541878C0B2461CF6B21E701823AB
:1024D00056E01878C0B2461CF6B21E70902616540C
:1024E0001878C0B2461CF6B21E702826165418780A
:1024F000C0B2461CF6B21E70042341E01878C0B288
:10250000461CF6B21E70902616541878C0B2461CAF
:10251000F6B21E70292616541878C0B2461CF6B2C0
:102520001E70B24B1B6815E01878C0B2461CF6B29C
:102530001E70902616541878C0B2461CF6B21E7053
:10254000FE2616541878C0B2461CF6B21E70A74B71
:102550001B685B082B4013E01878043816540426D7
:102560001878033816541878C0B2461CF6B21E709C
:10257000912616541878C0B2461CF6B21E70FF237E
:1025800001311354217073E30620944B944E197853
:10259000C9B24A1CD2B21A70924A50541978C9B2C0
:1025A000481CC0B21870052050541978C9B2481C94
:1025B000C0B21870002050541978C9B2481CC0B27B
:1025C00018703078C0B2441CE4B23470505419789A
:1025D000C9B2481CC0B21870902050541978C9B2C2
:1025E000481CC0B2187002A880795054292814D011
:1025F000FE2843D11978C9B2481CC0B21870022015
:1026000002ABDB795354794A116881431160591E3A
:102610008B4111685B00FFF7F4FB1978734CC9B26A
:10262000481CC0B2187002ABD87950542268AA4333
:102630002260236803432360FFF7ECF86C4B1A68B1
:102640002A431A602222DA60F82252025A601D617F
:10265000BFF36F8F1E69664F002EFBD15B21F82000
:1026600049424002FFF7E4F821686248FFF7E0F8CA
:102670003B68AB433B60604B5E60F9E21978C9B2DE
:10268000481CC0B21870002350E402AB9879534C38
:10269000032848D909212278514FD2B2531CDBB20A
:1026A0002370504B99542278D2B2511CC9B2217078
:1026B000082199542178C9B24A1CD2B22270002252
:1026C0005A542178C9B2481CC0B220703878C0B2C0
:1026D000461CF6B23E7058542178C9B2481CC0B2AC
:1026E0002070B82058542178C9B2481CC0B220705C
:1026F000FF2058542178C9B2481CC0B220705A54E7
:102700002178C9B2481CC0B220705A542178C9B28D
:10271000481CC0B220705A542178C9B2481CC0B2BB
:1027200020705A54A4E223782E4EDBB25A1CD2B247
:1027300022700922F2542378294FDBB25A1CD2B2FC
:1027400022700822F2542378DBB25A1CD2B22270D3
:102750000022F2542378DBB25A1CD2B222703A78AB
:10276000D2B2511CC9B23970F2542378DBB25A1C70
:10277000D2B22270B822F2542378DBB25A1CD2B201
:102780002270F05402ABDF79012F07D92378DBB236
:102790005A1CD2B22270FF22F25408E03900FDF731
:1027A000F1FC2378DBB25A1CD2B22270F7540B4BE7
:1027B00000201A78D2B2511CC9B219700221B1544A
:1027C0001A78D2B2511CC9B21970B0541A78D2B268
:1027D000511CC9B21970B0544AE2C0466C000020C6
:1027E0008402002084010020120000208C020020BE
:1027F00000C0005004F00100FC0000500920E64B2E
:1028000000241978E54FC9B24A1CD2B21A70E44AC2
:1028100050541978C9B2481CC0B2187008205054DE
:102820001978C9B2481CC0B2187054541978C9B28A
:10283000481CC0B218703878C0B2461CF6B23E7060
:1028400050541978C9B2481CC0B21870B8205054FE
:102850001978C9B2481CC0B2187002A886795654BB
:10286000D04908682840A04240D003207600B040FC
:10287000CD4F397801421CD11978C9B2481CC0B279
:102880001870FF2050541978C9B2481CC0B2187093
:10289000022050541978C9B2481CC0B21870802068
:1028A00050541978C9B2481CC0B218700623FFF7FB
:1028B0003DFB1878C0B2411CC9B21970397831415A
:1028C000294011541978C9B2481CC0B218700220AE
:1028D00050541978C9B2481CC0B2187054541978B1
:1028E000C9B2481CC0B218705454C1E11978C9B2B9
:1028F0004C1CE4B21C70FF2454541978C9B24C1C0F
:10290000E4B21C700224545412E40720A24BA34EDC
:102910001978C9B24A1CD2B21A70A14A5054197817
:10292000C9B2481CC0B21870062050541978C9B2F8
:10293000481CC0B21870002050541978C9B2481C05
:10294000C0B218703078C0B2441CE4B23470505435
:102950001978C9B2481CC0B21870B92050541978FF
:10296000C9B2481CC0B2187002A8847954541978AE
:10297000C079C9B2FE2800D0A4E0481CC0B21870CB
:10298000FE2050541978C9B2481CC0B2187002AB6E
:102990001B7A5354854A08211355854A1368FFF75B
:1029A00030FA07207C4B7D4E1978C9B24A1CD2B24E
:1029B0001A707B4A50541978C9B2481CC0B21870BA
:1029C000062050541978C9B2481CC0B218700020B3
:1029D00050541978C9B2481CC0B218703078C0B2CF
:1029E000441CE4B2347050541978C9B2481CC0B2C7
:1029F0001870B920505402A988791978C9B20328EF
:102A000060D800F0A5F902193148481CC0B218700E
:102A10000020505402A9C8791978C9B24C1CE4B2FC
:102A20001C70FE2851D150541978C9B2481CC0B24C
:102A300018705E4B1B7814E0481CC0B218705554D7
:102A400002A9C8791978C9B24C1CE4B21C70FE28DE
:102A50003BD150541978C9B2481CC0B21870534BBE
:102A60005B78DBB2FFF762FA481CC0B21870022034
:102A7000505402A9C8791978C9B24C1CE4B21C7030
:102A8000FE2822D150541978C9B2481CC0B218701F
:102A9000464B9B78E5E7481CC0B2187003205054A1
:102AA00002A9C8791978C9B24C1CE4B21C70FE287E
:102AB0000BD150541978C9B2481CC0B218703B4BA6
:102AC000DB78CEE74C1CE4B21C70FF24FFF735FB2B
:102AD00002AB9A79374B1A7002AAD2795A7002AABD
:102AE000127A9A7002AA527ADA70C1E0324902A8C8
:102AF0000B68407A1B0E984200D0B9E00B6802A820
:102B00001B0C807ADBB2984200D0B1E002A8C47AF4
:102B1000FF200B681B0A03409C4200D0A8E002ABD8
:102B200009681B7B0840834200D0A1E0802105207A
:102B3000136889040B431360174B184E1978C9B2F8
:102B40004A1CD2B21A70164A50541978C9B2481C9D
:102B5000C0B21870042050541978C9B2481CC0B2D1
:102B60001870002050541978C9B2481CC0B21870AF
:102B70003078C0B2441CE4B2347050541978C9B2F1
:102B8000481CC0B21870942050541978C9B2481C1F
:102B9000C0B2187055546BE06C0000208402002015
:102BA000840100208C0200207600002077000020A5
:102BB000AC020020480000201800002002AB9B79E6
:102BC000002B55D102AB5B7A3E2B51D1514902AA61
:102BD0000B68927A1B0E9A424AD102ABD87AFF2335
:102BE0000A68120C1A40904242D10A6802A8007B7F
:102BF000120A1A4090423BD102AA0968527B0B404C
:102C00009A4235D1FEF706FE0121434B1A680A436A
:102C10001A602222DA60F82252025A601961BFF368
:102C20006F8F1A693C4D002AFBD121783B4B09027A
:102C300019433B48FEF7FCFD03222B6813432B602E
:102C4000384A394B1A60FEE71A68002AFCD1374B24
:102C50001A70FEF7DFFD03212F4A13680B43136040
:102C6000304A314B1A60A022D20593682B439360FF
:102C700002AB9B78002B29D102AA1279042A20D01A
:102C8000092A07D0032A21D18021294AC9021368C1
:102C90000B431AE08020274A80051360244A1168FC
:102CA0000143116024490B7024490B7024490B70B7
:102CB00024490B7010682449014011601B4A1370AD
:102CC00004E01B4A204B11680B40136002AB1A78DA
:102CD0005B7801339A4210DDDBB2D21A02A90A7086
:102CE000002201320198D1B2884201D8FEF7BAFE23
:102CF00002A81918895C8154F3E70D4B134A19682F
:102D00000A4080211A601A6849040A431A6013B005
:102D1000F0BDC0461800002000C000503E00FFFF7C
:102D20001CF001000400FA050CED00E08402002014
:102D3000AC0200207C420050C10400206E00002044
:102D4000B2040020C2040020FFFFFBFFFFFFFFFBD7
:102D500002B4714649084900095C49008E4402BC2E
:102D60007047C046002243088B4274D303098B424C
:102D70005FD3030A8B4244D3030B8B4228D3030C4B
:102D80008B420DD3FF22090212BA030C8B4202D3ED
:102D90001212090265D0030B8B4219D300E0090A15
:102DA000C30B8B4201D3CB03C01A5241830B8B421E
:102DB00001D38B03C01A5241430B8B4201D34B0307
:102DC000C01A5241030B8B4201D30B03C01A52416C
:102DD000C30A8B4201D3CB02C01A5241830A8B42F1
:102DE00001D38B02C01A5241430A8B4201D34B02DA
:102DF000C01A5241030A8B4201D30B02C01A52413E
:102E0000CDD2C3098B4201D3CB01C01A52418309F1
:102E10008B4201D38B01C01A524143098B4201D32B
:102E20004B01C01A524103098B4201D30B01C01A56
:102E30005241C3088B4201D3CB00C01A52418308D0
:102E40008B4201D38B00C01A524143088B4201D3FD
:102E50004B00C01A5241411A00D20146524110465D
:102E60007047FFE701B5002000F006F802BDC0463C
:102E70000029F7D076E770477047C04670B50F2A33
:102E800032D90C0004430B00A40731D11500040013
:102E9000103D2D0901352D0149191E6826605E6817
:102EA00066609E68A660DE681033E6601034994262
:102EB000F3D10F2345191340032B1BD91C1F0023EB
:102EC000A4080134A400CE58EE5004339C42FAD139
:102ED00003232D1909191A4005D00023CC5CEC54AA
:102EE00001339A42FAD170BD0500002AF5D1FAE704
:102EF0000500F2E71A00F8E701020204001BB70020
:102F00000000000080F0FA0210270000000000001E
:0C2F1000000000000000000000805101E3
:0C2F1C0080F0FA0280F0FA02320000009F
:00000001FF
